:100000000C9434000C9451000C9451000C94510049
:100010000C9451000C9451000C9451000C9451001C
:100020000C9451000C9451000C9451000C9451000C
:100030000C9451000C9451000C9451000C945100FC
:100040000C9470010C9451000C9451000C945100CC
:100050000C9451000C9451000C9451000C945100DC
:100060000C9451000C94510011241FBECFEFD4E02A
:10007000DEBFCDBF11E0A0E0B1E0E8EBF6E002C0EA
:1000800005900D92A430B107D9F721E0A4E0B1E0CA
:1000900001C01D92A630B207E1F70E94E9010C945D
:1000A0005A030C940000809102019091030106977D
:1000B00009F441C086E090E090930301809302012F
:1000C00088E290E090930101809300018FE39CE926
:1000D0000197F1F700C00000409102015091030127
:1000E0006AE081E00E94C6029FEF23EC89E0915014
:1000F00020408040E1F700C0000084E190E0909350
:100100000101809300019FEF22E587E0915020409C
:100110008040E1F700C0000084EB90E09093010183
:10012000809300019FEF26E181E1915020408040C3
:10013000E1F700C00000089522988091020190919B
:100140000301039741F41A9B06C00E94C1020E945A
:1001500053000E94A702809102019091030102972F
:1001600059F41A9B09C00E94C10248E06AE081E08C
:100170000E94C6020E94A7024B992DC080910201E5
:1001800090910301029739F586E090E09093030186
:10019000809302012FEF81E19AE721508040904047
:1001A000E1F700C000002FEF81E19AE72150804085
:1001B0009040E1F700C000002FEF81E19AE7215065
:1001C00080409040E1F700C0000083E090E0909311
:1001D0000301809302010895CF930E94A70202C0F9
:1001E0000E949C000E94B4028111FACF0E94BC02BE
:1001F000882341F08A3031F0803F09F048C002C0C6
:100200000E949C000E94B4028111FACF0E94BC029D
:10021000C82F02C00E949C000E94B4028111FACF34
:10022000C130A9F50E94BC02843049F018F4813035
:10023000D9F41DC0853051F08730B1F40EC082E092
:1002400090E0909303018093020111C083E090E05D
:1002500090930301809302010AC00E94C1020E9490
:1002600053000E94A70213C00E94C10210C00E9446
:10027000C1028FE39CE90197F1F700C000004091B3
:100280000201509103016AE081E00E94C602CF9111
:10029000089514BC85E085BD88E586BD81E0809326
:1002A0006E00209A289A8FEA94E00197F1F700C037
:1002B000000080910001909101011816190674F454
:1002C00080E090E025E12A95F1F700000196209169
:1002D00000013091010182179307A4F32898089533
:1002E0001F920F920FB60F9211242F933F938F936B
:1002F0009F9388E586BD809102019091030102974A
:1003000079F48091040190910501C39794F19BB118
:1003100080E489278BB9109205011092040129C04D
:100320008091020190910301039779F48091040177
:10033000909105010697ECF09BB180E489278BB979
:10034000109205011092040114C080910201909155
:100350000301069771F480910401909105010297C1
:1003600044F09BB180E489278BB91092050110926B
:10037000040180910401909105010196909305017B
:1003800080930401209A289A8FEA94E00197F1F76C
:1003900000C000008091000190910101181619061B
:1003A00074F480E090E025E12A95F1F700000196D1
:1003B000209100013091010182179307A4F328983E
:1003C0009F918F913F912F910F900FBE0F901F9093
:1003D00018950E941E0280E296E00E945F0247E0AC
:1003E00060E081E00E94480280E895E20E946F028E
:1003F00066E080E00E9496020E944901569A539856
:100400005B9A78940E94EC00FDCF449840E120E094
:1004100030E0992314F4409A01C04098220F331F12
:1004200033992160419A880F991F00C000004198BC
:10043000415079F7449A822F932F089587B18361B1
:1004400087B9449A2FEF80E792E021508040904096
:10045000E1F700C0000080EE90EC0E94050287EDFD
:1004600090E80E9405028BEA92EC0E94050281E866
:100470009AEC0E94050280E090EE0E94050280E066
:1004800098EC0E94050287EF94EC0E940502089503
:10049000477050E05469637070E0660F771F660F15
:1004A000771F660F771F20E2829FC00111249927D2
:1004B000862B972B842B952B0E940502089580365E
:1004C000910538F080342FE0920728F08FE39FE009
:1004D00002C080E690E0906A0E9405020895873984
:1004E00022E0920710F1883125E1920780F49C0107
:1004F00040E050E060E678EA80E090E00E943E0351
:10050000C90101978068966C0E94050208959C01BC
:1005100040E050E06CEF72E485E090E00E941C0344
:10052000C9010197966C0E9405020895877090E0BA
:10053000986920E1629FB00111247727862B972BC1
:100540000E94050208954498339BFECF089588ECDD
:1005500092E80E94050281E89AEC0E94050283E875
:100560009AEC0E9405020895449886B183FB88277F
:1005700080F991E08927089580E090EB0E940502C0
:10058000089588E092E80E94050208951F93CF9392
:10059000DF93182FD62FC42F88E392E80E9405021C
:1005A0000E94A3028AEA98EB0E9405020E94A3021D
:1005B0008AEA98EB0E9405020E94A3028AEA98EB5D
:1005C0000E9405020E94A3028DE298EB0E940502A0
:1005D0000E94A30284ED98EB0E9405020E94A302F0
:1005E000812F90E0986B0E9405020E94A3028D2F3C
:1005F00090E0986B0E9405020E94A3028C2F90E06D
:10060000986B0E9405020E94A30280E098EB0E9472
:1006100005020E94A30288E092E80E9405022FEFE3
:1006200080E792E0215080409040E1F700C0000058
:10063000DF91CF911F910895A1E21A2EAA1BBB1B37
:10064000FD010DC0AA1FBB1FEE1FFF1FA217B3079E
:10065000E407F50720F0A21BB30BE40BF50B661FB4
:10066000771F881F991F1A9469F760957095809578
:1006700090959B01AC01BD01CF010895052E97FB1C
:1006800016F4009407D057FD0DD00E941C0307FC00
:1006900009D07EF490958095709561957F4F8F4F2E
:1006A0009F4F089550954095309521953F4F4F4F5E
:0806B0005F4F0895F894FFCF9D
:0406B800B400020088
:00000001FF
